:0400000084EF10F089
:1000080000C015F0E1CF16F0E2CF17F09EAA16D087
:10001800AECFCDF09E9A300E3C5C10E2CE0EE16E73
:10002800000EE26E3C50E126D8B0E22ACDC0E6FFD1
:100038003C2A300E3C5CD8B03C6A3A2A15C000F025
:0A00480016C0E1FF17C0E2FF11002F
:0C0052000E0E0D6E0D2EFED700001200E9
:10005E0040C304F041C305F03EC302F03FC303F0BA
:10006E0042C300F043C301F0010E0301425F000ED4
:10007E00435B005001100FE004C0E9FF05C0EAFF2A
:10008E0002C0E1FF03C0E2FFEECFE6FF024A032A01
:10009E00044A052AE5D73EC300F03FC301F0120023
:0600AE009D8A9D981200DE
:0600B4009D9A9D981200C8
:1000BA000301386B396B376B3651000808E135514B
:1000CA00000805E13451000802E13351375D7AE254
:1000DA003A0E3E6F030E3F6F38C300F0000E016EFA
:1000EA0000360090013600360090013600502F2568
:1000FA00406F01503021416F040E426F000E436F72
:10010A00A9DF39513125E16E000E3221E26E000E6F
:10011A003A15056EFF0E3B15066E3CC307F03DC34C
:10012A0008F0000E0716081606C000F007C001F016
:10013A0008C002F0036A00C0E6FF392B39513125A5
:10014A00E16E000E3221E26EFF0E3A15006E00C01B
:10015A00E6FF392B39513125E16E000E3221E26E6C
:10016A00000E3A15056E000E3B15066E000E3C1584
:10017A00076EFF0E3D15086E08C000F0016A026A9C
:10018A00036A00C0E6FF392B39513125E16E000EB2
:10019A003221E26E000E3A15056E000E3B15066E10
:1001AA00FF0E3C15076E000E3D15086E07C000F0E5
:1001BA0008C001F0026A036A00C0E6FF392B382B37
:0601CA00372B7AD712006A
:1001D000066A076A056A33C301F034C302F035C307
:1001E00003F036C304F001360190023603360436BC
:1001F0000450000808E10350000805E1025000081F
:1002000002E10150055C13E2075003013125E16E64
:10021000000E3221E26E06502F25E96E000E3021CD
:10022000EA6EEECFE6FF072A062A052AD4D7120087
:100230000A6A0B6A096A03013651000808E1355160
:10024000000805E13451000802E13351095CD8B0DF
:10025000A1D00B503125E16E000E3221E26E0AC0B2
:1002600000F0000E016E003600900136003600905E
:10027000013600502F25E96E01503021EA6EFF0E45
:10028000EE14006E00C0E6FF0B2A0B503125E16E24
:10029000000E3221E26E0AC000F0000E016E003640
:1002A0000090013600360090013600502F25E96E8F
:1002B00001503021EA6E000EEE14056EFF0EEE14B2
:1002C000066EEECF07F0EECF08F0000E0716081608
:1002D00006C000F007C001F008C002F0036A00C0C9
:1002E000E6FF0B2A0B503125E16E000E3221E26E43
:1002F0000AC000F0000E016E003600900136003694
:100300000090013600502F25E96E01503021EA6E31
:10031000000EEE14056E000EEE14066EFF0EEE14C7
:10032000076E000EEE14086E07C000F008C001F062
:10033000026A036A00C0E6FF0B2A0B503125E16E0A
:10034000000E3221E26E0AC000F0000E016E00368F
:100350000090013600360090013600502F25E96EDE
:1003600001503021EA6E000EEE14056E000EEE1400
:10037000066E000EEE14076EFF0EEE14086E08C037
:1003800000F0016A026A036A00C0E6FF0B2A0A2A2B
:06039000092A51D71200FA
:10039600066A076A056A03013651000808E1355105
:1003A600000805E13451000802E13351055C3BE2E7
:1003B60007503125E16E000E3221E26E06C000F0D4
:1003C600000E016E00360090013600502F25E96EB2
:1003D60001503021EA6E000EEE14036EEE50FF0B54
:1003E600046E04C000F0016A00C0E6FF072A075049
:1003F6003125E16E000E3221E26E06C000F0000EDD
:10040600016E00360090013600502F25E96E01502E
:100416003021EA6EFF0EEE14006E00C0E6FF072ADA
:08042600062A052AB8D71200CE
:10042E0042DE000E006E03013251005C02E13151DA
:10043E003A5C04E23AC031F3000E326F336B346B28
:10044E003251345D02E13151335D18E233512F25C3
:10045E00E16E34513021E26ECE0EE96E000EEA6E80
:10046E003B50E926D8B0EA2AEECFE6FF3B2A300E03
:10047E003B5CD8B03B6A334B342BE2D731513A5EFA
:0C048E000FDE31C300F032C301F0120099
:10049A000CDE3AC02FF3000E0301306F03DE2FC3C8
:0804AA0000F030C301F0120064
:1004B2000301356B366B376B386B33C300F034C3D3
:1004C20001F001320032019E01320032019E0132FE
:1004D2000032019E00C005F0070E3315016E34C3D1
:1004E20002F0000E0216000E021802E1000E0118C0
:1004F200D8A4052A066A0550065C46E20650312554
:10050200E16E000E3221E26EE66A076A080E075CAF
:1005120039E206503125036E000E3221046E2F514E
:100522003525E96E30513621EA6EEECF02F007C072
:1005320001F002C000F0015004E000360090FF0F0D
:10054200FBD703C0E9FF04C0EAFFEE50001203C06C
:10055200E1FF04C0E2FF00C0E6FF010E3527000EF6
:10056200362337233823000E385D08E1000E375D4D
:1005720005E13451365D02E13351355D01E304D0CA
:0A058200072AC4D7062AB7D71200D3
:10058C00C26A070EC012C08E2FC300F00036009056
:10059C00003600900050C212C28055DDC282C2A249
:1005AC0001D0FDD7C4CF01F0006AC3500012000E79
:0605BC000112C2901200C2
:1005C200036A046A056A000E006E03013451005C7E
:1005D20002E13351055C32E2010E076E066A080E33
:1005E200065C2AE204503125E16E000E3221E26EF1
:1005F20003502F25E96E000E3021EA6E0750EE14EB
:10060200026E06C001F002C000F0015004E00032A8
:10061200009EFF0FFBD700C0E6FF042A07360790B3
:10062200052A000E006E3451005C02E13351055C74
:0E06320001E304D0062AD3D7032AC5D712004D
:100640000301386B396B376B3651000808E13551BF
:10065000000805E13451000802E13351375D51E2F1
:100660003A6B3B6B3C6B3D6B38512F25E96E000EAE
:100670003021EA6EEECF01F001C03BF33A6B3C6BE8
:100680003D6B000E3C6F3D6F382B38512F25D96ED6
:10069000000E3021DA6EDE503A13000E3B133C138D
:1006A0003D13382B382B38512F25E96E000E3021A1
:1006B000EA6EEECF03F0006A016A00503A1301506F
:1006C0003B13000E3C133D13382B39C300F0000ED2
:1006D000016E003600900136003600900136005061
:1006E00031253E6F015032213F6F3A0E406F030EAD
:1006F000416F040E426F000E436FB1DC392B372B74
:04070000A3D7120069
:10070400076A086A066A03013651000808E1355190
:10071400000805E13451000802E13351065CD8B009
:100724009CD008C000F0000E016E00360090013627
:1007340000360090013600503125E16E015032211F
:10074400E26E07502F25E96E000E3021EA6EEECFDF
:10075400E6FF000EE66EE66EE66E072A08C000F0BD
:10076400000E016E0036009001360036009001360E
:1007740000503125046E01503221056E07502F259B
:10078400E96E000E3021EA6EEECF03F003C001F0F3
:10079400006A04C0E9FF05C0EAFF000E026E036EA2
:1007A400EE500012EE500112EE500212EE500312FF
:1007B40004C0E1FF05C0E2FF00C0E6FF01C0E6FFA0
:1007C40002C0E6FF03C0E6FF072A08C000F0000EDF
:1007D400016E00360090013600360090013600505C
:1007E4003125046E01503221056E07502F25E96E24
:1007F400000E3021EA6EEECF03F0006A016A04C0F5
:10080400E9FF05C0EAFF000E026E036EEE5000120F
:10081400EE500112EE500212EE50031204C0E1FF3A
:1008240005C0E2FF00C0E6FF01C0E6FF02C0E6FF2C
:1008340003C0E6FF072A08C000F0000E016E003670
:1008440000900136003600900136315100263251B5
:0C0854000122072A082A062A56D71200A3
:10086000066A076A056A33C301F034C302F035C370
:1008700003F036C304F00136019002360336043625
:100880000450000808E10350000805E10250000888
:1008900002E10150055C13E2075003013125E16ECE
:1008A000000E3221E26E06502F25E96E000E302137
:1008B000EA6EEECFE6FF072A062A052AD4D71200F1
:1008C000056A066A046A03013651000808E13551D9
:1008D000000805E13451000802E13351045C4DE2A7
:1008E00006C000F0000E016E003600900136005088
:1008F0003125E16E01503221E26E05502F25E96E5F
:10090000000E3021EA6EEECF03F003C001F0006A62
:1009100000C0E6FF01C0E6FF06C000F0000E016E59
:1009200000360090013600503125026E0150322110
:10093000036E0550010F006E016A000E0122005087
:100940002F25D96E01503021DA6E02C0E9FF03C0B5
:10095000EAFFDE50EE10006EEECF01F0000E011245
:1009600002C0E1FF03C0E2FF00C0E6FF01C0E6FFF6
:0C097000062A020E0526042AA6D7120053
:0A097C00000EACB2010E006E120076
:100986005AEC00F03A6A3B6A3C6A196A186A57ECF4
:0409960000F012005B
:10099A008FD1030128512625016E29512721026E84
:1009AA00000E006E0250005C02E10150100802E2E3
:1009BA00066A02D0010E066E9DD103012851262532
:1009CA00016E29512721026E000E006E0250005C52
:1009DA0002E10150100802E2066A02D0010E066E18
:1009EA0089D10301000E275D02E1000E265D1BE39B
:1009FA00000E006E2751005C02E12651090813E33C
:100A0A0028512625016E29512721026E000E006EFB
:100A1A000250005C02E10150140802E2066A02D0A8
:100A2A00010E066E7DD0000E275D02E1140E265DD2
:100A3A0021E3000E006E2751005C02E126511D08D9
:100A4A0019E3140E265D006E000E2759016E285117
:100A5A000024026E29510120036E000E006E03501D
:100A6A00005C02E102500A0802E2066A02D0010EA4
:100A7A00066E56D0000E275D02E1280E265D21E3A0
:100A8A00000E006E2751005C02E12651310819E37D
:100A9A00280E265D006E000E2759016E285100248B
:100AAA00026E29510120036E000E006E0350005C95
:100ABA0002E102500A0802E2066A02D0010E066E3C
:100ACA002FD0000E275D02E13C0E265D28E3000EC2
:100ADA00006E2751005C02E126513F0820E33C0EDC
:100AEA00265D046E000E2759056E28C300F029C33F
:100AFA0001F000360090013600500424026E0150C5
:100B0A000520036E000E006E0350005C02E10250E5
:100B1A00080802E2066A02D0010E066E01D0066AD1
:100B2A00E9D028512625016E29512721026E000E8F
:100B3A00006E0250005C02E10150140802E2066AEB
:100B4A0002D0010E066ED6D028512625016E2951F3
:100B5A002721026E000E006E0250005C02E1015075
:100B6A00100802E2066A02D0010E066EC3D0000E19
:100B7A00275D02E1000E265D1BE3000E006E275181
:100B8A00005C02E12651090813E328512625016E6B
:100B9A0029512721026E000E006E0250005C02E10C
:100BAA000150140802E2066A02D0010E066E7DD0D8
:100BBA00000E275D02E1140E265D21E3000E006E91
:100BCA002751005C02E126511D0819E3140E265D27
:100BDA00006E000E2759016E28510024026E295119
:100BEA000120036E000E006E0350005C02E1025009
:100BFA000A0802E2066A02D0010E066E56D0000EFC
:100C0A00275D02E1280E265D21E3000E006E2751C2
:100C1A00005C02E12651310819E3280E265D006EB8
:100C2A00000E2759016E28510024026E2951012015
:100C3A00036E000E006E0350005C02E102500A08C7
:100C4A0002E2066A02D0010E066E2FD0000E275D60
:100C5A0002E13C0E265D28E3000E006E2751005C7F
:100C6A0002E126513F0820E33C0E265D046E000E89
:100C7A002759056E28C300F029C301F000360090F9
:100C8A00013600500424026E01500520036E000E46
:100C9A00006E0350005C02E10250080802E2066A94
:100CAA0002D0010E066E01D0066A24D0066A22D04E
:100CBA0003012551010AD8B46CD62551020AD8B4C9
:100CCA007CD62551030AD8B48CD62551040AD8B447
:100CDA0028D72551050AD8B437D725510F0AD8B4D1
:100CEA0033D72551060AD8B442D72551100AD8B4A9
:0A0CFA003ED7DCD706C000F0120060
:100D0400010E03012E6F010E2C6F000E2D6F800E4D
:100D1400006E800E2D19005C02E12C51140821E3B1
:100D24004DEC02F00050011001E01BD0000E2D1913
:100D340002E1140E2C1908E12AC3E1FF2BC3E2FFE0
:100D4400040EE66E006A26D0030E0C6E970E0D6E2E
:100D54000D2EFED70C2EFCD7000000002C4B2D2BA3
:100D6400D6D728C32FF329C330F324C331F325C3C3
:100D740032F317EC02F026C3E1FF27C3E2FF00C001
:100D8400E6FF01C0E6FF2AC3E1FF2BC3E2FFE66AE8
:060D94002EC300F0120066
:100D9A00FF0E0101016FFF0E026FFF0E036FFF0EC0
:100DAA00046FFF0E0D6FFF0E0E6F000E0F6F000E19
:100DBA00106FFF0E056FFF0E066F000E076F000E15
:100DCA00086F7C0E096F090E0A6F000E0B6F000E7A
:100DDA000C6FAC8A900EAB6E948E949C9EAA03D034
:080DEA00AECF00F0FBD71200B0
:100DF200E7D02AC32FF32BC330F31A0E03012625A3
:100E0200316F000E2721326F28C333F329C334F325
:100E1200E1EC02F0E6D0000E0301275D02E1000ED4
:100E2200265D22E3000E006E2751005C02E126518E
:100E320009081AE32AC32FF32BC330F326C300F0A9
:100E420027C301F0003600900136650E0024316F91
:100E5200000E0120326F28C333F329C334F3000E8E
:100E6200356F366F2CDDABD0000E275D02E1140E1C
:100E7200265D39E3000E006E2751005C02E1265127
:100E82001D0831E32AC32FF32BC330F3140E265D62
:100E9200016E000E2759026E01C003F002C004F079
:100EA20004320332049E03C000F004C001F0003695
:100EB20000900136003600900136510E0024316F49
:100EC200000E0120326F28C333F329C334F3000E1E
:100ED200356F366F34333333349F000E356F366FD0
:100EE20020EC03F06CD0000E275D02E1280E265D97
:100EF20039E3000E006E2751005C02E126513108F1
:100F020031E32AC32FF32BC330F3280E265D016E83
:100F1200000E2759026E01C003F002C004F0043231
:100F22000332049E03C000F004C001F000360090BA
:100F320001360036009001363D0E0024316F000E5E
:100F42000120326F28C333F329C334F3000E356F07
:100F5200366F34333333349F000E356F366F82EC85
:100F620003F02DD0000E275D02E13C0E265D27E343
:100F7200000E006E2751005C02E126513F081FE37C
:100F82002AC32FF32BC330F33C0E265D036E000EF3
:100F92002759046E03C000F004C001F0003600902F
:100FA2000136C50E0024316F000E0120326F28C3B6
:100FB20033F329C334F3000E356F366F50DC11D092
:100FC20003012551050AD8B414D725510F0AD8B404
:100FD20010D72551060AD8B41ED72551100AD8B405
:060FE2001AD7006A12009C
:100FE800010E03012F6FC6EC02F015D11A0E030192
:100FF80026252F6F000E2721306F2AC331F32BC30C
:1010080032F328C333F329C334F359EC02F013D174
:101018002A0E26252F6F000E2721306F2AC331F3A1
:101028002BC332F328C333F329C334F359EC02F04A
:1010380002D1000E275D02E1000E265D23E3000EBB
:10104800006E2751005C02E1265109081BE326C304
:1010580000F027C301F0003600900136650E002429
:101068002F6F000E0120306F2AC331F32BC332F3E8
:1010780028C333F329C334F3000E356F366FCBEC36
:1010880001F0ACD0000E275D02E1140E265D39E3B5
:10109800000E006E2751005C02E126511D0831E365
:1010A800140E265D016E000E2759026E01C003F072
:1010B80002C004F004320332049E03C000F004C0EE
:1010C80001F0003600900136003600900136510ECE
:1010D80000242F6F000E0120306F2AC331F32BC379
:1010E80032F328C333F329C334F3000E356F366F58
:1010F80034333333349F000E356F366F5DEC00F0B8
:101108006DD0000E275D02E1280E265D39E3000E42
:10111800006E2751005C02E12651310831E3280EA8
:10112800265D016E000E2759026E01C003F002C051
:1011380004F004320332049E03C000F004C001F03E
:101148000036009001360036009001363D0E00242E
:101158002F6F000E0120306F2AC331F32BC332F3F7
:1011680028C333F329C334F3000E356F366F343395
:101178003333349F000E356F366F18EC01F02ED0E4
:10118800000E275D02E13C0E265D28E3000E006E8E
:101198002751005C02E126513F0820E33C0E265D02
:1011A800036E000E2759046E03C000F004C001F05E
:1011B800003600900136C50E00242F6F000E012066
:1011C800306F2AC331F32BC332F328C333F329C357
:1011D80034F3000E356F366FE8EC00F02CD026C3E0
:1011E80000F027C301F00036009001369D0E002460
:1011F80003012F6F000E0120306F2AC331F32BC378
:1012080032F328C333F329C334F3000E356F366F36
:10121800CBEC01F010D003012551010AD8B4E6D671
:101228002551020AD8B4F4D62551030AD8B401D7F7
:0A1238002551040AD4E0006A1200F8
:10124200020E03011525E96E000E1621EA6EEECF9D
:1012520001F001C01BF31A6B030E1525D96E000EA7
:101262001621DA6EDE501A13000E1B13040E15251A
:10127200E96E000E1621EA6EEECF03F003C001F014
:10128200006A00C01CF301C01DF3050E1525D96EBE
:10129200000E1621DA6EDE500010026E01C003F05D
:1012A200000E031202C01CF303C01DF3000E035C08
:1012B20002E1010E025CD8A080D0000E006E1D512A
:1012C200005C02E11C514008D8A077D015C3E9FFA9
:1012D20016C3EAFFEECF23F314C324F3010E152540
:1012E200E96E000E1621EA6EEECF25F31AC326F33D
:1012F2001BC327F31CC328F31DC329F3CDEC04F051
:101302000050010A56E115C3E9FF16C3EAFFEECF0A
:1013120023F314C324F3010E03011525E96E000E15
:101322001621EA6EEECF25F31AC326F31BC327F369
:101332001CC328F31DC329F3030E17252A6F000EC1
:1013420018212B6F50DE00C019F30050000A2DE166
:10135200010E03011725E16E000E1821E26E010E47
:101362001525E96E000E1621EA6EEECFE6FF020E9B
:101372001725E16E000E1821E26E1CC300F0003644
:10138200009000C0E6FFFB0E1725E16E000E18214B
:10139200E26E020E1725E96E000E1821EA6E020EA9
:1013A200EE24006E00C0E6FF03D00301040E196FA5
:1013B20003D00301020E196F02D0030E196F19C375
:0413C20000F0120025
:1013C600410E0C6EEE0E0D6E0D2EFED70C2EFCD7BA
:0C13D6000000C3EC04F0010E006E1200D9
:1013E2000F013A6BB886B06ACF0EAF6EAC84D4DC14
:1013F200020E0B6E040E0C6EBA0E0D6E0D2EFED783
:101402000C2EFCD70B2EFAD70000F28CF28E57EC82
:0414120000F01200D4
:1014160003011B6B14C323F317C324F318C325F36B
:10142600190E266F030E276F15C328F316C329F36B
:101436001B0E2A6F030E2B6F62DC0050000A03E1BD
:101446001BC300F014D0154B162B1951175D016EF6
:101456001A511859026E01C017F302C018F3000E94
:10146600021802E1000E0118D5E11BC300F01200BC
:101476000301206B010E216F000E226F020E15254F
:10148600E96E000E1621EA6EEECF01F001C01FF3E1
:101496001E6B030E1525D96E000E1621DA6EDE5070
:1014A6001E13000E1F13010E1525E96E000E1621E0
:1014B600EA6EEE500F0A67E1040E1525E96E000E7E
:1014C6001621EA6EEECF03F003C001F0006A00C0F9
:1014D60021F301C022F3050E1525D96E000E162143
:1014E600DA6EDE500010026E01C003F0000E031229
:1014F60002C021F303C022F3000E035C02E1010ED9
:10150600025C0BE3000E006E2251005C02E12151E9
:10151600400803E3010E006E01D0006A005203E1A9
:10152600030E206F2FD021C300F022C301F0013239
:101536000032019E01320032019E01320032019ECC
:1015460000C01AF3070E2115016E22C302F0000E29
:101556000216000E021802E1000E0118D8A41A2B7A
:10156600060E1525D96E000E1621DA6E1A51DE18F2
:1015760003E0030E206F06D0070E15251C6F000E24
:1015860016211D6F2FD0040E1525E96E000E1621AB
:10159600EA6EEE50000A0BE1050E1525E96E000E07
:1015A6001621EA6EEE50000A02E11B6B17D0040EFC
:1015B6001525E96E000E1621EA6EEE50FF0A0CE1C3
:1015C600050E1525E96E000E1621EA6EEE50000A8C
:1015D60003E1010E1B6F02D0030E206F1B0E1C6F62
:1015E600030E1D6F2051000A67E115C3E9FF16C3FC
:1015F600EAFFEECF23F314C324F3010E1525E96E9B
:10160600000E1621EA6EEECF25F31EC326F31FC386
:1016160027F321C328F322C329F3CDEC04F00050AD
:10162600010A47E115C3E9FF16C3EAFFEECF23F32C
:1016360014C324F3010E03011525E96E000E1621CD
:10164600EA6EEECF25F31EC326F31FC327F321C38D
:1016560028F322C329F31CC32AF31DC32BF3F9EC89
:1016660006F000C020F30050000A1FE1010E03013E
:10167600196F1951050810E319511725E16E000E6F
:101686001821E26E19511525E96E000E1621EA6E33
:10169600EECFE6FF192BEDD7FB0E1725E16E000EF8
:1016A6001821E26E050EE66E03D00301040E206FCC
:0E16B60003D00301020E206F20C300F01200CB
:1016C40003011C6B040E1D6F010E1E6F000E1F6FB5
:1016D400020E1525E96E000E1621EA6EEECF01F01A
:1016E40001C01BF31A6B030E1525D96E000E1621CB
:1016F400DA6EDE501A13000E1B13010E1525E96E67
:10170400000E1621EA6EEE50100A51E1040E152562
:10171400E96E000E1621EA6EEECF03F003C001F06D
:10172400006A00C01EF301C01FF3050E1525D96E13
:10173400000E1621DA6EDE500010026E01C003F0B6
:10174400000E031202C01EF303C01FF3000E035C5D
:1017540002E1010E025C0BE3000E006E1F51005CFF
:1017640002E11E51400803E3010E006E01D0006A3D
:10177400005203E1030E1C6F1AD01EC302F01FC3F4
:1017840003F0023602900336060E1525D96E000EBC
:101794001621DA6EDECF01F0000E031802E10150CB
:1017A400021803E0030E1C6F02D0070E1D6F1C51BC
:1017B400000A69E115C3E9FF16C3EAFFEECF23F37C
:1017C40014C324F3010E1525E96E000E1621EA6EEA
:1017D400EECF25F31AC326F31BC327F31EC328F346
:1017E4001FC329F3CDEC04F00050010A49E115C3ED
:1017F400E9FF16C3EAFFEECF23F314C324F3010E6B
:1018040003011525E96E000E1621EA6EEECF25F3CD
:101814001AC326F31BC327F31EC328F31FC329F3DC
:101824001D5115252A6F000E16212B6FF9EC06F0B9
:1018340000C01CF30050000A1FE1010E0301196FE0
:101844001951050810E319511725E16E000E1821EE
:10185400E26E19511525E96E000E1621EA6EEECFDF
:10186400E6FF192BEDD7FB0E1725E16E000E1821AC
:10187400E26E050EE66E03D00301040E1C6F03D066
:0C1884000301020E1C6F1CC300F01200D8
:10189000FF0E0301176FFF0E186FFB0E1525E96E83
:1018A000000E1621EA6EEE50010F006E016A000E66
:1018B000012200C005F0046A0550045C2DE20450CA
:1018C0001525D96E000E1621DA6EDE501819026E3B
:1018D000036A000E031A000E036E380E0224F66E21
:1018E000220E0320F76E000EF86E000EF82209009B
:1018F000F5CF00F000501719186F380E0224F66E5D
:10190000210E0320F76E000EF86E000EF82209007B
:10191000F5CF17F3042AD0D705501525E16E000E38
:101920001621E26E18C3E6FF0550010F006E016A32
:10193000000E012200501525E16E01501621E26EC5
:0619400017C3E6FF1200D0
:10194600949082800301186B000E006E1751005CA4
:1019560002E11651185D10E2BEEC04F00050000AD8
:1019660001E1FAD718511425E96E000E1521EA6E29
:10197600EECFADFF182BE8D7BEEC04F00050000AFE
:1019860001E1FAD7829018C300F0000E016E120032
:10199600020E03011525E96E000E1621EA6EEECF42
:1019A60001F001C01BF31A6B030E1525D96E000E4C
:1019B6001621DA6EDE501A13000E1B13040E1525BF
:1019C600E96E000E1621EA6EEECF03F003C001F0B9
:1019D600006A00C01CF301C01DF3050E1525D96E63
:1019E600000E1621DA6EDE500010026E01C003F002
:1019F600000E031202C01CF303C01DF3000E035CAD
:101A060002E1010E025CD8A0ABD0000E006E1D51A3
:101A1600005C02E11C514008D8A0A2D015C3E9FF22
:101A260016C3EAFFEECF23F314C324F3010E1525E4
:101A3600E96E000E1621EA6EEECF25F31AC326F3E1
:101A46001BC327F31CC328F31DC329F3CDEC04F0F5
:101A56000050010AD8A480D015C3E9FF16C3EAFFD7
:101A6600EECF23F314C324F3010E03011525E96E0B
:101A7600000E1621EA6EEECF25F31AC326F31BC31A
:101A860027F31CC328F31DC329F3030E17252A6F5A
:101A9600000E18212B6FF4EC07F000C019F300506C
:101AA600000A56E1010E03011725E16E000E18210A
:101AB600E26E010E1525E96E000E1621EA6EEECFD6
:101AC600E6FF020E1725E16E000E1821E26E1CC31A
:101AD60000F01DC301F001320032019E01320032D6
:101AE600019E01320032019E00C0E6FF070E1C1562
:101AF600016E1DC302F0000E0216000E021802E16E
:101B0600000E011813E0020E1725016E000E1821B3
:101B1600026E01C0E9FF02C0EAFFEE50010F006E3F
:101B260001C0E1FF02C0E2FF00C0E6FFFB0E172581
:101B3600E16E000E1821E26E020E1725E96E000E08
:101B46001821EA6E020EEE24006E00C0E6FF03D0F6
:101B56000301040E196F03D00301020E196F02D0A0
:0A1B6600030E196F19C300F01200FE
:101B70000101006B0BC314F3010E03010C25156F5B
:101B8000000E0D21166F010E176F000E186F43DC4B
:101B900000C000F10050000A01E0ACD0010E0C259D
:101BA000126F000E0D21136F37D00301040E106F5A
:101BB000000E116F020E0E6F000E0F6F66D0030144
:101BC0000BC314F3020E0C25156F000E0D21166FBA
:101BD000050E176F000E186F1EDC00C000F10050DC
:101BE000000A11E1060E0C25E96E000E0D21EA6EC9
:101BF000EECF10F3000E116F000E116F070E0E6F77
:101C0000000E0F6F00D041D00A0E0101006F0BC310
:101C100014F3E3EC09F039D012C3E9FF13C3EAFF70
:101C2000EE50010AC2E012C3E9FF13C3EAFFEE500F
:101C3000020ABBE012C3E9FF13C3EAFFEE50030A36
:101C4000B4E012C3E9FF13C3EAFFEE50040AADE0AB
:101C500012C3E9FF13C3EAFFEE50050AA6E012C360
:101C6000E9FF13C3EAFFEE50060A9FE012C3E9FF43
:101C700013C3EAFFEE500F0AA2E012C3E9FF13C339
:101C8000EAFFEE50100A9BE0BFD701010051000AA5
:101C900031E1000E006E03011151005C02E11051B0
:101CA000FB0808E2080E0101006F0BC314F3E3EC1C
:101CB00009F020D00BC314F303010E510C25156F4E
:101CC0000F510D21166F10C317F311C318F30BEC4E
:101CD0000AF000C000F10050000A00E0FB0E0C25E5
:101CE000E16E000E0D21E26E10510E25006E000611
:0A1CF00000C0E6FF00C100F0120082
:101CFA0003010B51010A03E1010E006E01D0006AD3
:021D0A001200C5
:101D0C00FF0E0101006FFF0E03010E6FFB0E0C2581
:101D1C00E96E000E0D21EA6EEE50010F006E016AA5
:101D2C00000E012200C007F0066A0750065C32E282
:101D3C0006500C25D96E000E0D21DA6EDE500E19F0
:101D4C00026E036A000E031A000E046E056E000E7E
:101D5C00036E046E056E380E0224F66E220E0320FE
:101D6C00F76E000E0420F86E0900F5CF00F000505D
:101D7C000101001903010E6F380E0224F66E210EBC
:101D8C000320F76E000E0420F86E0900F5CF00F169
:101D9C00062ACBD707500C25D96E000E0D21DA6E12
:101DAC000E51DE1813E10750010F006E016A000E90
:101DBC00012200500C25D96E01500D21DA6E010163
:101DCC000051DE1803E1010E006E01D0006A120012
:101DDC00010E0101006F10C314F311C315F30CC3F2
:101DEC0016F30DC317F3A9DD0EC3E1FF0FC3E2FF1A
:101DFC0000C0E6FF01C0E6FF12C3E1FF13C3E2FF20
:081E0C00E66A00C100F01200BB
:061E1400010E006E120039
:0A1E1A00F1EC09F0010E006E120059
:101E24000101006B010E03010C25106F000E0D2142
:101E3400116F3ED00BC314F30CC315F30DC316F38B
:101E44000EC317F30FC318F3A4DD00C000F169D06B
:101E54000BC314F30CC315F30DC316F30EC317F31E
:101E64000FC318F321EC09F000C000F15AD00BC3E2
:101E740014F30CC315F30DC316F30EC317F30FC3FA
:101E840018F33BEC0AF000C000F14BD00BC314F381
:101E94000CC315F30DC316F30EC317F30FC318F3D6
:101EA4000FDC00C000F13DD0010E0101006F39D0FC
:101EB40010C3E9FF11C3EAFFEE50010ABBE010C3EF
:101EC400E9FF11C3EAFFEE50020AB4E010C3E9FFD0
:101ED40011C3EAFFEE50030ABBE010C3E9FF11C3CC
:101EE400EAFFEE50040AB4E010C3E9FF11C3EAFFAD
:101EF400EE50050ABCE010C3E9FF11C3EAFFEE503F
:101F04000F0AB5E010C3E9FF11C3EAFFEE50060A59
:101F1400BDE010C3E9FF11C3EAFFEE50100AB6E0BA
:101F2400C3D701010051000A22E0010E03010E256E
:101F3400E16E000E0F21E26E010E0C25E96E000E1B
:101F44000D21EA6E800EEE10006E00C0E6FF020E58
:101F54000E25E16E000E0F21E26E00C1E6FFFB0EBE
:101F64000E25E16E000E0F21E26E020EE66E0CC32A
:101F7400E9FF0DC3EAFFEECF00F00EC3E1FF0FC38C
:101F8400E2FF00C0E6FF0BC314F30EC315F30FC347
:081F940016F37CDC006A120068
:041F9C003EDF120012
:101FA0000900F5CFE6FF0006FBE10106F9E11200AA
:041FB00031DF12000B
:061FB4004DEC02F01200EA
:101FBA000001FF6BFEC014F3110E0301156F010E31
:101FCA00166F010E176F000E186F0BEC0AF000C0A7
:101FDA00FFF00050000A01E08FD011C10BF3FEC0E0
:101FEA000CF386DE0050010A05E001011151000AD6
:101FFA0001E07BD0FEC00BF3110E03010C6F010E42
:10200A000D6FB1DD00C0FFF00050000A05E00001CD
:10201A00FF510A0A01E068D00001FF51000A2DE1D0
:10202A00FEC014F302010C51010F006E016A000E8A
:10203A000122110E00240301156F010E0120166FF3
:10204A00020E176F000E186F0BEC0AF000C0FFF0BB
:10205A000050000A01E011D0FEC00BF3110E0C6F04
:10206A00010E0D6F4EDE0050010A07E0070E000157
:10207A00FF6FFEC014F3E3EC09F00001FF51000A00
:10208A0004E0FF510A0A01E02FD0FF51000A00E1E3
:10209A00FEC00BF3110E03010C6F010E0D6F0D0E36
:1020AA000E6F020E0F6FB9DE01011151000A1CE01A
:1020BA00020E030108250C6F0D6B000E0D230C4B4D
:1020CA000D2BFEC00BF3090E0E6F030E0F6F0D0ED4
:1020DA00106F020E116FFF0E126F000E136F79DE72
:1020EA000050000A01E100D007D0060E0001FF6F80
:0E20FA00FEC014F3E3EC09F0FFC000F012008A
:10210800F7EC11F0020E0F01386F44DF0050010A9E
:102118000DE10001FE6B4ADF000E015C02E1080ED2
:10212800005C03E30001FE6B44DFF3D73DDFFFD71C
:1023EE0010EE18F0B50E006E010E016E380EF66E80
:0E23FE00230EF76E000EF86ED0EC0FF01200FA
:1021380000C0C101C30302C2C60607C705C5C4045F
:10214800CC0C0DCD0FCFCE0E0ACACB0BC90908C8CF
:10215800D81819D91BDBDA1A1EDEDF1FDD1D1CDCBF
:1021680014D4D515D71716D6D21213D311D1D0102F
:10217800F03031F133F3F23236F6F737F53534F41F
:102188003CFCFD3DFF3F3EFEFA3A3BFB39F9F8388F
:1021980028E8E929EB2B2AEAEE2E2FEF2DEDEC2C7F
:1021A800E42425E527E7E62622E2E323E12120E0EF
:1021B800A06061A163A3A26266A6A767A56564A4DF
:1021C8006CACAD6DAF6F6EAEAA6A6BAB69A9A8684F
:1021D80078B8B979BB7B7ABABE7E7FBF7DBDBC7C3F
:1021E800B47475B577B7B67672B2B373B17170B0AF
:1021F800509091519353529296565797559594549F
:102208009C5C5D9D5F9F9E5E5A9A9B5B995958980E
:10221800884849894B8B8A4A4E8E8F4F8D4D4C8CFE
:10222800448485458747468682424383418180406E
:1022380000C1814001C0804101C0804100C181408E
:1022480001C0804100C1814000C1814001C080417E
:1022580001C0804100C1814000C1814001C080416E
:1022680000C1814001C0804101C0804100C181405E
:1022780001C0804100C1814000C1814001C080414E
:1022880000C1814001C0804101C0804100C181403E
:1022980000C1814001C0804101C0804100C181402E
:1022A80001C0804100C1814000C1814001C080411E
:1022B80001C0804100C1814000C1814001C080410E
:1022C80000C1814001C0804101C0804100C18140FE
:1022D80000C1814001C0804101C0804100C18140EE
:1022E80001C0804100C1814000C1814001C08041DE
:1022F80000C1814001C0804101C0804100C18140CE
:1023080001C0804100C1814000C1814001C08041BD
:1023180001C0804100C1814000C1814001C08041AD
:1023280000C1814001C0804101C0804100C181409D
:0123380000A4
:0123390000A3
:10233A00000001010000000001010101000100018B
:10234A00010100000101010100000000010001007B
:01235A000082
:01235B000081
:01235C000080
:10235D004E61BC00817051011DC80602D367510149
:04236D0066FFEE55C4
:10237100A4704582B81E638452780B87B84E758865
:0423810048E10384A8
:1023850001110222033304440555066607770888C0
:1023950009990AAA000000000000000000000000E2
:0823A500000000000000000030
:1023AD0043747220726561636865642032300A007F
:1023BD0002220444066608880AAA01110333055552
:1023CD0007770999000000000000000000000000E0
:0823DD000000000000000000F8
:0823E500434F4C574159000021
:020000040030CA
:0D000100221F3CFFBF81FF0FC00FE00F402A
:00000001FF
